:020000040000FA
:040000008301D92877
:08000800A000030EA100851900
:100010000D282C090000851510282C0885111028A2
:10002000831281000B11210E8300A00E200E090007
:1000300082070034013401340234023403340434BE
:1000400004340534053406340634073407340834E0
:10005000093409340A340A340B340B340C340C34AC
:100060000D340E340E340F340F3410341034113478
:100070001134123412341334133414341434153448
:100080001534163416341734173418341834193418
:1000900019341A341A341B341B341B341C341C34EA
:1000A0001D341D341E341E341E341F341F342034BE
:1000B0002034213421342134223422342234233494
:1000C000233424342434243425342534253426346C
:1000D0002634273427342734283428342834293444
:1000E0002934293429342A342A342A342B342B3421
:1000F0002B342C342C342C342D342D342D342D34FD
:100100002D342D342408A2070318A50A2508A307B7
:10011000003422082402A20003188F28A30A23080F
:100120002502A30000342208260203189C28031984
:100130009C280130A6000034A601003423082502C3
:100140000319A928031CB2280319B2280130A600FC
:10015000003422082402031CB2280319B2280130FB
:10016000A6000034A601003422082602031DBB2885
:100170000130A6000034A6010034A3013608A20015
:100180000310A20DA30DA60BC0282208B307030875
:100190000139B2072308B2070034B5013708B302AA
:1001A0000318D728B20803190800B20BD728B50ADC
:1001B000CF28831203309F00831607308500860105
:1001C000831286018316D230810083128B178B161F
:1001D0003230AC00B101B0019930AF00AD01AE01D9
:1001E00005290E30A200A20BF32800001F1F0729CB
:1001F0000608AD000A290E30A200A20BFD2800005F
:100200009F1F11290608AE0014298312860183124C
:10021000860FF128831286010E30A200A20B0E2950
:1002200000008312860FFB2883122D08A8002F08D8
:10023000A6002808A200932083122608261C422923
:100240002D08A8002F082802B6002E08A8002F08A5
:10025000A6002808A200932083122608261C38290D
:100260002E08A8002F082802B7000130AA00402954
:1002700083122F08A8002E082802B7000230AA0017
:100280008312642983122F08A8002D082802B600C3
:100290002E08A8002F08A6002808A2009320831289
:1002A0002608261C5B292E08A8002F082802B70064
:1002B0000430AA00632983122F08A8002E08280200
:1002C000B7000330AA00831283123608A80037084B
:1002D000A6002808A200932083122608261C79294C
:1002E0000130AB003608B4003708B6003408B70058
:1002F0007C2983120230AB008312B301B2010310D8
:100300000630A600BD200530A600BD200230A600A4
:10031000BD20CD2035081820B100B0012A08A80062
:100320000430A6002808A200B42083122608261C48
:10033000BB292B08A8000130A6002808A200B42081
:1003400083122608261CBA295A30A2000030A300C6
:100350002208A8002308A9003108A2003008A30041
:100360002908A5002808A400892083122208B100CA
:100370002308B000831283122A08A8000330A600C5
:100380002808A200B42083122608261C012A2B0864
:10039000A8000130A6002808A200B4208312260875
:1003A000261CE9295A30A2000030A3002208A80028
:1003B0002308A9003108A2003008A3002908A500DD
:1003C0002808A400822083122208B1002308B0006C
:1003D000002A8312B430A2000030A3002208A80033
:1003E0002308A9003108A2003008A3002908A500AD
:1003F0002808A400892083122208B1002308B00035
:10040000831283122A08A8000230A6002808A2003E
:10041000B42083122608261C472A2B08A800013086
:10042000A6002808A200B42083122608261C2F2A22
:100430000E30A2000130A3002208A8002308A90062
:100440003108A2003008A3002908A5002808A4004C
:10045000892083122208B1002308B000462A8312A3
:10046000B430A2000030A3002208A8002308A9008D
:100470003108A2003008A3002908A5002808A4001C
:10048000822083122208B1002308B0008312831255
:100490002A08A8000130A6002808A200B420831270
:1004A0002608261C8D2A2B08A8000130A600280843
:1004B000A200B42083122608261C752A0E30A20042
:1004C0000130A3002208A8002308A9003108A200D7
:1004D0003008A3002908A5002808A4008220831260
:1004E0002208B1002308B0008C2A83126830A200D1
:1004F0000130A3002208A8002308A9003108A200A7
:100500003008A3002908A5002808A4008920831228
:100510002208B1002308B000831283120310B00C2C
:0A052000B10C32303107AC000529A0
:00000001FF
